:100000000C9462000C94B51A0C94E21A0C948A00B9
:100010000C948A000C948A000C948A000C948A0038
:100020000C948A000C948A000C948A000C948A0028
:100030000C948A000C948C0B0C948A000C948A000B
:100040000C940F1B0C948A000C948B1E0C94CE1EE7
:100050000C948A000C948A000C948A000C948A00F8
:100060000C94ED080C948A000000000700020100C7
:100070000003040600000000000000000102040864
:100080001020408001020408102001020408102002
:10009000040404040404040402020202020203032E
:1000A00003030303000000002300260029000000D2
:1000B0000000250028002B0000000000240027007D
:1000C0002A00422011241FBECFEFD8E0DEBFCDBFF3
:1000D00012E0A0E0B1E0E8EFF2E402C005900D927A
:1000E000AA3CB107D9F714E0AAECB2E001C01D9216
:1000F000A43BB107E1F710E0C4ECD0E004C02297C4
:10010000FE010E945721C23CD107C9F70E947E2000
:100110000C947A210C9400008091B603813019F47C
:1001200082E08093B6038091B603833019F484E0B3
:100130008093B6030895A8950895CF93DF93FC01AB
:10014000962F9270862F817060FF20C0992331F026
:100150008091480380831092CA0216C0A091CA02FF
:10016000C091E103C770D0E0CA56DD4F8881A8175F
:1001700010F080E03CC081E08A0F8093CA02B0E0BA
:10018000A850BD4F8C91808381E031C09923C1F08C
:1001900090819093CB021092CA02292F207E2036A4
:1001A00051F490914803923020F390819F71909385
:1001B0008A0393E01AC09E3F39F71092480317C094
:1001C0009091CB029F3F01F79091CA02993288F635
:1001D00021E0290F2093CA023081E92FF0E0E75493
:1001E000FC4F3083293281F691E090934803DF91F0
:1001F000CF910895DC01ED91FC910190F081E02D0B
:1002000009950895DC01ED91FC910190F081E02DBC
:10021000099508952091B7033091B803382748E035
:10022000C901880F991F37FF06C09C0151E225279D
:1002300050E1352701C09C01415091F73093B8033C
:100240002093B70308958436910520F4BC0180E023
:1002500090E017C09C018E3B910528F42A55310986
:10026000AAE0B0E00CC0823D910528F4245B31097E
:10027000A4E6B0E004C02D5C3109A8E5B2E00E941C
:100280008B20A4E6B0E09B01AC010E949A20089567
:1002900090E08C599F4F0E942301089587E080933E
:1002A000E20380E28093E30381E28093E40310920F
:1002B000E50386E28093E6038093E70384E280937C
:1002C000E80385E28093E903089560E089E00E94F5
:1002D0001D1C61E088E00E941D1C61E087E00E9417
:1002E0001D1C60E082E00E941D1C61E084E00E9411
:1002F0001D1C089542E050E06CE870E080E00E9430
:10030000951A0895E3E0F0E089E080935700E491C6
:10031000E67081E0E63009F080E00895CF93DF9346
:10032000C82F0E948201882381F0DFB781E080938B
:10033000B503F8940E949B0088E180936000C0930D
:100340006000C1110E949B00DFBFDF91CF91089533
:10035000FC0140A5842F877090E0959587950196C4
:10036000242F217030E0820F931F880F880F08958B
:100370008F929F92AF92BF92CF92DF92EF92FF92B5
:10038000CF93FC01C0A5EC2FE770F0E0EA56FD4FDB
:10039000A081B0E0C7FF03C024E130E002C02FE03D
:1003A00030E0FC0197A183E1989FF0011124E65A07
:1003B000FE4F80809180A280B380A20FB31F20E403
:1003C0003FE14DE750E00E94A520A50194010E9465
:1003D000DD208C2F887149F469017A01E0EDCE0EA1
:1003E000E7E0DE1EE11CF11C1BC0C7FF05C060E496
:1003F0007AE88CE29EE004C060E07EEE8AEB9BE04F
:1004000069017A01F8EBCF0EFBE0DF1EE11CF11C65
:10041000A50194010E94DD20C20ED31EE41EF51E2C
:10042000C701B60169517C4F8F4F9F4F28EE33E0D3
:1004300040E050E00E94DD20A8EEB3E00E949A2048
:10044000CF91FF90EF90DF90CF90BF90AF909F90B3
:100450008F900895DB01FA01582F569590E0248182
:10046000237030E0322F22274081240F311D119656
:100470003C932E9344814C70218130E060E4469F90
:10048000200D311D112413963C932E931297448115
:100490004073228130E060E1469F200D311D112420
:1004A00015963C932E9314974481407C238130E031
:1004B00064E0469F200D311D112417963C932E9326
:1004C0001697359618969F5F591748F680FF47C0D4
:1004D000408142954695469543702DE431E0429F18
:1004E000C001439F900D11240C9611969C938E93FE
:1004F000808190E074E0969587957A95E1F7837016
:100500009927829FA001839F500D929F500D112427
:10051000445F5F4F13965C934E931297808190E0F7
:10052000969587959695879583709927829FA001C8
:10053000839F500D929F500D1124445F5F4F15967D
:100540005C934E93149740814370429FC001439F38
:10055000900D11240C9617969C938E9316970895E0
:10056000803223E0920708F1883E23E0920740F4AE
:100570008F519340E4E096958795EA95E1F70895C9
:10058000803D27E0920718F48C5D934008958839E8
:1005900028E0920768F4885C974074E09695879508
:1005A0007A95E1F78D509C4F089580E090E0089592
:1005B0008FEF93E008958C30910540F4A4E0880F0C
:1005C000991FAA95E1F7885D9C4F0895843F23E029
:1005D000920718F484529C4F0895811524E09207E5
:1005E00040F48657934FF4E0880F991FFA95E1F78E
:1005F000089580E998E008959C0136952795257522
:100600003575821B930B9C012373337396958795E5
:100610009695879583739373820F931F9C0154E083
:10062000369527955A95E1F7280F391F2F703F709F
:1006300041E051E0249FC001259F900D349F900D13
:100640001124892F08955F98882319F00000289AB3
:1006500002C00000289800005F9A000008955F9A89
:10066000000083B15F980000869581700895CF9354
:10067000DF93D82F5C9A5F985C98C8E08D2F8078C4
:100680000E942303DD0FC150C9F75F98DF91CF911E
:1006900008958F770E9437030895CF93DF93D82F63
:1006A000C8E08D2F80780E942303DD0FC150C9F769
:1006B0005F98DF91CF910895CF93DF935F98C8E063
:1006C00080E0D82FDD0F0E942F038D0FC150C9F796
:1006D000DF91CF9108950E9449030E945C035C9AC8
:1006E0000895A1E0B0E0E7E7F3E00C942E218068E4
:1006F00069830E9437036981862F0E944D035C9AAB
:100700002196E2E00C944A21CF93C091C203C827FE
:10071000E82FF0E0E754FC4F678589E70E947103FA
:100720006C2F8DE30E9471036C2F82E40E94710391
:10073000CF91089586E20E946B030895CF938BE2D8
:100740000E946B03C82F8CE20E946B03282F30E0BD
:1007500066E0369527956A95E1F744E0C49FC001AD
:100760001124822B932BCF910895CF93DF93EC012B
:100770006C818CE10E9471036D818DE10E94710397
:100780006E818EE10E9471036F8180E20E9471038D
:10079000688581E20E947103698582E20E9471038B
:1007A0006A8583E20E9471036B8584E20E94710373
:1007B0006C8585E20E9471036D858AE20E94710357
:1007C0006E858EE60E9471036F858FE60E9471032D
:1007D000688980E70E947103698981E70E9471033B
:1007E0006A8982E70E947103DF91CF910895CF92C9
:1007F000DF92EF92FF92CF93DF936B017C01C114E4
:1008000088E3D8068CE9E8068CE1F80628F5C701EC
:10081000B60120E836E948E950E00E94DD20E90110
:10082000689760E879E687E69FEF0E94AD206C0D3F
:100830007D1D8E1D9F1DF2E0660F771F881F991F7B
:10084000FA95D1F721E732E040E050E00E94DD2048
:10085000F22EE32E80E421C0C701B60120E03DE284
:1008600041E351E00E94DD20E901689760E073ED0B
:100870008EEC9EEF0E94AD206C0D7D1D8E1D9F1D88
:10088000660F771F881F991F21E732E040E050E094
:100890000E94DD20F22EE32E80E66C2F6F71680F30
:1008A00085E70E9471036E2D86E70E9471036F2D0C
:1008B00087E70E947103DF91CF91FF90EF90DF9067
:1008C000CF9008958F929F92AF92BF92CF92DF9276
:1008D000EF92FF92CF93DF93D82F83E00E946B03B8
:1008E0008093B40384E00E946B038093B30360E0C1
:1008F00086E00E94710361E087E00E9471036FE768
:1009000089E00E94710365E08AE00E94710362E160
:100910008BE00E94710365E18CE00E9471036DEF32
:100920008DE00E94710360E08EE00E947103DD2380
:1009300019F087E491E008C02091E00333E1239FA0
:10094000C0011124865A9E4F0E94B5036CE880E3D3
:100950000E9471036FE082E30E94710362E483E30B
:100960000E9471038091E10387FF02C064E101C02E
:100970006AE084E30E9471036AE285E30E947103E6
:100980006DE286E30E94710364ED87E30E947103C8
:1009900060E088E30E94710360E089E30E947103D4
:1009A000D11109C0C090C203D090C303E090C4032A
:1009B000F090C50307C0C5E9CC2EC1ECDC2EED2CB0
:1009C000CEEDFC2ECAE38F2C9924AA24BB24682DDB
:1009D0008C2F0E947103682D85E08C0F0E9471039B
:1009E000FE2CED2CDC2CCC24CF5FCE3361F76FEFE7
:1009F00083E40E9471036FEF84E40E9471036FEF40
:100A000085E40E9471036FEF86E40E947103DD2389
:100A100011F066E002C06091C6038DE60E9471038A
:100A200060E089E70E9471036091C7038AE70E9432
:100A3000710360E083E70E94710360E084E70E9435
:100A40007103D11109C06091BE037091BF03809101
:100A5000C0039091C10304C060E071EA8CEB93E3A2
:100A60000E94F703DF91CF91FF90EF90DF90CF903E
:100A7000BF90AF909F908F90089561E087E00E94B3
:100A8000710364E28EE70E94710363E088E00E94D4
:100A9000710360E088E00E94710365E087E00E94D6
:100AA000710362E085E00E94710383E00E946B03A2
:100AB0008093B40384E00E946B038093B303089592
:100AC00083E00E946B038093B40384E00E946B0375
:100AD0008093B30361E087E00E9471036AE070E0F5
:100AE00080E090E00E94881B0E943D050000089570
:100AF000CF92DF92FF920F931F93CF93DF931F92BA
:100B0000CDB7DEB7082F162F8EE399830E947103AD
:100B1000F02EC02E9981D92E8C2D8F19811738F483
:100B2000F60161916F018FE70E947103F5CF64E0D8
:100B300085E00E94710383E00E946B038093B403FD
:100B400084E00E946B038093B3030E94651B609353
:100B5000AF037093B0038093B1039093B20369E045
:100B600087E00E94710381E08093B6030F90DF91CC
:100B7000CF911F910F91FF90DF90CF9008950F9329
:100B80001F930E9478058091B603813099F40E94EA
:100B9000651B0091AF031091B0032091B103309118
:100BA000B203601B710B820B930B603A7648814055
:100BB000910548F38091B603813031F46AEB71E01E
:100BC0008AE094E00E94271D1F910F9108950F93D2
:100BD0001F938091B603823021F41092B60381E016
:100BE00020C08091B6038130D9F40E94651B00912A
:100BF000AF031091B0032091B1033091B203601B99
:100C0000710B820B930B613A76488140910540F05D
:100C100061E087E00E9471031092B60382E001C098
:100C200080E01F910F910895EF92FF920F931F9311
:100C3000CF93DF938B019C01442737FD4095542FC0
:100C400060E271EA87E090E00E94FF20E9011C1653
:100C50001D0614F0C1E0D0E0D80120E231EA47E0FF
:100C600050E00E94A5209E01442737FD4095542F57
:100C70000E94FF20790100E010E00E151F055CF4D2
:100C8000289ACE010E94AE1B2898CE010E94AE1B6E
:100C90000F5F1F4FF2CFCDB7DEB7E6E00C944621D1
:100CA000CF93DF932C9A6091F2037091F3038091BC
:100CB000F4039091F5030E94F70360E089E70E9436
:100CC000710361E070E080E090E00E94881B0E9468
:100CD0009A03C82F61E070E080E090E00E94881BDA
:100CE0000E949A03D0E0C80FD11D61E070E080E05F
:100CF00090E00E94881B0E949A03C80FD11D61E0FA
:100D000070E080E090E00E94881B0E949A032C987B
:100D10009E01280F311DC901969587959695879557
:100D2000DF91CF910895CF93C82F2C9A83E00E9432
:100D30006B038093B40384E00E946B038093B3033E
:100D400060E086E00E94710361E087E00E94710329
:100D50006FE789E00E94710365E08AE00E947103F9
:100D600062E18BE00E94710365E18CE00E947103F7
:100D70006DEF8DE00E94710360E08EE00E947103D0
:100D80006CE280E70E94710360E080E30E947103DF
:100D900060E089E70E94710365E08AE70E947103C1
:100DA00062E181E70E94710362E082E70E947103C1
:100DB00060E083E70E94710360E084E70E947103B2
:100DC0006091F2037091F3038091F4039091F50325
:100DD0000E94F70367E08DE60E9471036AE070E00D
:100DE00080E090E00E94881B69E087E00E94710328
:100DF0006AE070E080E090E00E94881BCC2369F0FC
:100E0000C5E1C15009F459C061E070E088EB91E0A0
:100E10000E9414060E949B00F4CF61E070E088E815
:100E200091E00E9414060E949B0065E08DE60E94FE
:100E300071036AE070E080E090E00E94881B61E04E
:100E400070E088EB91E00E9414060E949B0064E031
:100E50008DE60E9471036AE070E080E090E00E94FD
:100E6000881B61E070E08DE591E00E9414060E940D
:100E70009B0062E08DE60E9471036AE070E080E012
:100E800090E00E94881B61E070E08FEA90E00E9491
:100E900014060E949B0060E08DE60E9471036AE0E8
:100EA00070E080E090E00E94881B62E070E085E0E6
:100EB00091E00E9414060E949B0061E087E00E947E
:100EC00071032C98CF910895CF93DF93EC014AE002
:100ED00050E06D2F70E08AE094E00E94EC1D6EE21D
:100EE0008AE094E00E940B1DBE0184E07695679530
:100EF0008A95E1F76F7077274AE050E08AE094E046
:100F00000E94EC1D6EE28AE094E00E940B1DBE017F
:100F10006F7077274AE050E08AE094E00E94EC1D71
:100F2000DF91CF910895D82FC0E0CD1780F42D9A8E
:100F300064E670E080E090E00E94881B2D9864E6F3
:100F400070E080E090E00E94881BCF5FEECF6CE203
:100F500071E080E090E00E94881BE6CF0F931F9322
:100F6000CF93DF93EC01062F15E0115051F0CE0125
:100F70000E946421081741F0602FCE010E946C216D
:100F8000F4CF82E00E949307DF91CF911F910F91E0
:100F90000895A0E0B0E0EFECF7E00C942021482E9B
:100FA000562EC0E0D0E0612C712CE12CF12C00E039
:100FB00010E0442079F081E04816A1F092E0491257
:100FC00019C028E4622E712C30E2E32EF12C0BE4E0
:100FD00013E010C0612C712C6BE1E62EF12C02EEB7
:100FE00013E008C04DE1642E712C59E2E52EF12C7E
:100FF00009EB13E043018C0E9D1E1092B803109272
:10100000B7033401A62CA818B12CC30101966C01BA
:10101000AE14BF04A8F4A00EB11E511006C0C30147
:101020000E946421F501808305C0F5016081C30140
:101030000E94AE07F50180810E940A013601E2CFCD
:10104000C301511018C0C3010E946421B82EC6010B
:101050000E9464212B2D30E0322F2227282B8091F3
:10106000B7039091B8038217930779F4C0E0D0E0FA
:10107000552453949ECF36016091B8030E94AE0769
:101080006091B703C6010E94AE07D395C13093E0CB
:10109000D90708F48ECF852DCDB7DEB7E0E10C94EB
:1010A0003C2160E081E00E94C907882331F081E0A3
:1010B0009091B903983309F080E0089561E081E0F0
:1010C0000E94C907089561E082E00E94C90708955F
:1010D00060E082E00E94C907811108C0EBE4F3E000
:1010E0001192119283E0EB36F807D1F70895A1E051
:1010F000B0E0EDE7F8E00C942E2189830E944E01C8
:1011000092E09093F0039FEF9093F1039AE0909315
:10111000FA031092FB031092FC031092F203109258
:10112000F3031092F4031092F5032EE12093F603DB
:101130009093F70328EB3BE03093F9032093F803F7
:101140008981882371F061E080E00E94C907EBE4A7
:10115000F3E01192119283E0EB36F807D1F70E9489
:1011600063082196E2E00C944A2160E080E00E944E
:10117000C907811103C081E00E9477080895CF93C9
:10118000C1E0811101C0C0E06C2F82E10E94561CB9
:101190006C2F83E10E94561C1092A9031092A803A1
:1011A0008091B9008C6F8093B90080E28093B80081
:1011B00085E48093BC00CF91089585ED8093BC00B9
:1011C0008091BC0084FDFCCF0895ECEBF0E0108230
:1011D00085E480831092A80308951F920F920FB6A2
:1011E0000F9211242F933F934F935F936F937F93AD
:1011F0008F939F93AF93BF93EF93FF93CF93DF931F
:101200001F92CDB7DEB78091B900887F803609F490
:10121000C7C0A8F5883209F464C098F4803109F495
:101220005DC038F4882309F4F3C0883009F456C04F
:10123000F1C0883109F455C0803209F0EBC082E07A
:10124000A7C0803409F477C078F4803309F45FC014
:10125000883309F0DFC084E08093A7038091A8035E
:101260008B7F8093A803D0C0803509F452C08835A5
:1012700009F467C0883409F0CDC085E089C0883999
:1012800009F4C0C0A8F4883709F48AC038F4883655
:1012900009F486C0803709F483C0BCC0883809F4DB
:1012A000B1C0803909F47FC0803809F0B3C07BC079
:1012B000803B09F493C038F4803A09F48CC0883A32
:1012C00009F48CC0A7C0803C09F49EC0883C09F496
:1012D0009BC0883B09F09EC080E081C08091AC0338
:1012E00013C08091A9039FEF980F9093A9038823BF
:1012F000D1F1E091AA03F091AB03CF010196909355
:10130000AB038093AA0380818093BB007DC083E000
:101310003FC0E091AA03F091AB03CF0101969093F7
:10132000AB038093AA038091BB0080838091A903C3
:1013300081508093A9038091A903823008F064C092
:1013400061C0E091AA03F091AB03CF0101969093A5
:10135000AB038093AA038091BB0080838091A90393
:1013600081508093A9038091A8038B7F8093A80369
:101370008091A80380FF4CC08091A8038E7F80934A
:10138000A8038091A80382608093A80384EA3DC0EB
:101390008093A7038091A8038B7F8093A80338C014
:1013A0001092A90331C0E091AD03F091AE033097E4
:1013B00049F18091BB0089838091A90391E0980F46
:1013C0009093A903811102C062E001C060E0CE01E8
:1013D0000196099515C00E94DD0816C081E0E091D4
:1013E000AD03F091AE03309769F0882311F063E00C
:1013F00001C061E0CE010196099599819093BB00EF
:10140000811102C085E801C085EC8093BC0002C058
:101410000E94DD080F90DF91CF91FF91EF91BF9176
:10142000AF919F918F917F916F915F914F913F917C
:101430002F910F900FBE0F901F9018958F929F9233
:10144000AF92BF92CF92DF92EF92FF92CF93DF9352
:10145000EC010E94651B6B017C014E01A12CB12C9B
:101460008091A80382FF11C02097D1F30E94651BD1
:101470006C197D098E099F0986169706A806B9067C
:1014800078F70E94E50881E004C08091A7031092DC
:10149000A703DF91CF91FF90EF90DF90CF90BF90A7
:1014A000AF909F908F900895A2E0B0E0EAE5FAE057
:1014B0000C942A21182F7B01022F047022FD05C0F5
:1014C00080910B0190910C0102C080E090E02A8392
:1014D00049830E941E0A2A814981811136C01092D7
:1014E000A7034093A903F092AB03E092AA03110F64
:1014F0001093AC039091A80321FF02C085E001C0C6
:1015000084E0892B8093A8038091A80381FF0BC0FE
:101510008091A8038D7F8093A8038091AC03809372
:10152000BB0085EC01C085EE8093BC00822F8170EA
:1015300020FF0BC0011105C080910B0190910C019F
:1015400002C080E090E00E941E0A2296E6E00C9421
:101550004621A2E0B0E0EFEAFAE00C942A21182F2D
:101560007B01022F047022FD05C080910B01909138
:101570000C0102C080E090E02A8349830E941E0A89
:101580002A814981811138C01092A7034093A90391
:10159000F092AB03E092AA03812F880F81608093C1
:1015A000AC039091A80321FF02C085E001C084E054
:1015B000892B8093A8038091A80381FF0BC08091A1
:1015C000A8038D7F8093A8038091AC038093BB0018
:1015D00085EC01C085EE8093BC00822F817020FFD6
:1015E0000BC0011105C080910B0190910C0102C04C
:1015F00080E090E00E941E0A2296E6E00C944621CC
:10160000A0E0B0E0E6E0FBE00C9428210E94651B1E
:101610000091A3031091A4032091A5033091A60388
:101620006B017C01C01AD10AE20AF30A9701860114
:1016300041E1C41647E2D406E104F10408F442C0D3
:101640002091A20331E0320F3093A20320FF02C0A9
:1016500017E001C010E06093A3037093A40380938C
:10166000A5039093A60363E070E08AE094E00E94F3
:10167000020161E070E08AE094E00E94020107E06C
:10168000010F812F90E0EC01CC0FDD1FC35FDE4F17
:1016900068817981672F772763707727880F991F73
:1016A000880F991F682B792B8AE094E00E94FA003A
:1016B0006881798177278AE094E00E94FA001F5FB1
:1016C0001013DFCFCDB7DEB7E8E00C94442125B18D
:1016D00090E0FC01EE0FFF1FE80FF91FEE5EFC4FDC
:1016E0008081282B25B988B19181892B88B98BB14C
:1016F0009281892B8BB9089585B190910F0389232D
:1017000085B988B190911003892388B98BB19091E4
:10171000110389238BB908951F920F920FB60F9270
:1017200011242F933F934F935F936F937F938F93E6
:101730009F93AF93BF93CF93EF93FF93C0916E03AB
:1017400080910601C81708F03EC080910D0390916A
:101750000E039093870080938600EC2FF0E0EE0F4D
:10176000FF1FE35FFE4F808191810E94DB02880FA3
:10177000991F90930E0380930D0380910D03909118
:101780000E032091070130910801281B390B30937B
:101790000801209307018091F8039091F903880FC5
:1017A000991F2817390720F49093080180930701A7
:1017B00080916C03811142C08091F00380FF41C091
:1017C000C830E0F53EC080910D0390910E039093D8
:1017D0008700809386008091070190910801909383
:1017E0000E0380930D0380916C03882319F08FEF13
:1017F0009FEF06C080910D0390910E038855924093
:1018000090938B0080938A0080E49CE99093080178
:101810008093070180918400909185008097D0F398
:101820000E947C0B80916D03811105C0809106019F
:1018300081500E94670B10926E0327C08FEF9FEFBD
:1018400006C080910D0390910E03885592409093AD
:101850008B0080938A00809184009091850080970E
:10186000D0F30E947C0B80916D03811104C08091A4
:101870006E03811106C080916E038F5F80936E03AB
:1018800004C081500E94670BF6CFFF91EF91CF917A
:10189000BF91AF919F918F917F916F915F914F9188
:1018A0003F912F910F900FBE0F901F90189524E03D
:1018B000829FC00111248C30910538F0853F23E0D0
:1018C000920728F084EF93E008958CE090E008956B
:1018D000CF93DF93C091F103C03390F48C2F8073CA
:1018E00039F0803141F480916F038295807F05C08B
:1018F0008091740302C080917503CF70D0E015C051
:10190000CF33E0F4CF70D0E080916F038295807F79
:101910000E94570CDE01AA0FBB1FA35FBE4F11969A
:101920009C938E932196809175030E94570CFE0123
:10193000EE0FFF1FE35FFE4F91838083DF91CF9116
:10194000089580917003909171039F770E94FC022B
:1019500080936F038F3029F48091750386958058AA
:1019600004C099E0899F802D112480937403F8941A
:101970000E94680C78948091E4038132E1F48091B4
:1019800074039FEF980F9E3F78F08091B0008F7D99
:101990008093B00061E080917403811101C060E028
:1019A00083E00E94561C08958093B4008091B0009B
:1019B00080628093B0000895FF920F931F93CF939E
:1019C000DF9303EE13E0C0E0D0E0B3E0FB2E8C2FFA
:1019D000D801ED918D019E2F907F9031F1F4EF7041
:1019E000F0E0EE0FFF1FE35FFE4F208131816F2D8E
:1019F0000E94BD20E92FF0E0EE0FFF1FE057FD4FE2
:101A000061E0808191818217930708F060E0FE0118
:101A1000E256FD4F80810E94561C2196C730D105A9
:101A2000B1F6CDB7DEB7E5E00C9447210F931F93D5
:101A3000CF93DF930BE413E0C0E0D0E02091F103FB
:101A4000822F8F7090E0C817D907E9F00196C81768
:101A5000D90711F42033B8F4F801808191819F7087
:101A6000892B79F0F894F801808191819F700E9410
:101A7000B002FE01EE0FFF1FE35FFE4F91838083F4
:101A800078940E94DC0C21960E5F1F4FC031D10567
:101A9000A9F6DF91CF911F910F910895FF920F93B7
:101AA0001F93CF93DF9389EB93E00E94A80180936B
:101AB00006019091F103292F2F70281304C081E0B3
:101AC000820F8093060190539F3060F4409106018D
:101AD00030E0842F90E001972817390719F44F5F01
:101AE0004093060180910601813118F080E18093D6
:101AF0000601E4E1F3E0DF0112971C92DF01119788
:101B00001C921082339683E0E932F807A1F74FEF79
:101B10003FEFA7EAB2E003EE13E02FEFE80189916F
:101B20008E018031F8F490E0FD0132976081FC0174
:101B3000EE0FFF1FE80FF91FEE5EFC4F8081862B32
:101B40008083CD010197EC0158818181852B8183B0
:101B50009C918281892B8283609550959095292351
:101B6000352346231396D3E00A3E1D07B9F640936A
:101B70000F033093100320931103CEE9D2E003EE5C
:101B800013E0F12CF80181918F01823230F086321E
:101B9000B8F0863211F460E010C0F5E0FF1204C026
:101BA0008091C1008F7E06C086E0F81205C080914A
:101BB000C100877F8093C10061E088810E941D1C65
:101BC000F3942196E7E0FE12DDCF8091E3038032AB
:101BD00031F461E08AE00E94561C82E201C082E09A
:101BE0008093800081E080936D0380936C038091EB
:101BF000E403813211F08732D9F461E083E00E947E
:101C00001D1C60E083E00E94561C8091E403813239
:101C100031F481E08093B0008093B10009C082E08C
:101C20008093B00085E08093B1008EE38093B30091
:101C30008AE1809381008FEF9FEF90938B008093D8
:101C40008A0080ED97E0909387008093860080E47F
:101C50009CE9909308018093070190930E03809371
:101C60000D0310926E0380916F00816080936F006E
:101C70008091F00383FF0DC080914B0390914C0342
:101C80009F70892B31F00E94160D10926C031092F8
:101C90006D03CDB7DEB7E5E00C944721CF93C82F95
:101CA0008091E5038B3221F46C2F8EE00E94561C4C
:101CB0008091E403873249F48091B000CC2311F085
:101CC000806101C08F7E8093B000CF910895A2E221
:101CD000B0E0EDE6FEE00C941E216B017C010E9459
:101CE000591B4B015C0181E00E94620483E08093F8
:101CF000B6030E94600566EC71E08AE094E00E9401
:101D0000271D7BE1272EE0E53E2EF7E47F2EA6E49B
:101D10004A2EB5E55B2EC114D104E104F10469F04B
:101D20000E94591B681979098A099B096C157D0560
:101D30008E059F0510F080E0D5C08091B6038430F9
:101D400051F764ED71E08AE094E00E94271D8FE76F
:101D50000E9449030E945C038AA3823601F509EBC5
:101D600013E00E945C03D8018D938D01B3E0023E25
:101D70001B07B9F78091B903883309F0ADC06DED49
:101D800071E08AE094E00E94271D82E48AA361E06A
:101D9000CE0182960E94BF052C9A81E0A3C08037B5
:101DA00041F0893611F581E00E94770889E4898342
:101DB00004C03982C12CD12C76019091B503809159
:101DC000F003992311F0806801C08F778093F003AE
:101DD000E2EEF3E0DE011296822D01900D928A95DB
:101DE000E1F76CE1CE01019675C08437E1F4E4E5DA
:101DF000E98383E08A8388E88B8387E08C838DE0A6
:101E00008D838AE1EDE2F1E0DE01169601900D92FC
:101E10008A95E1F76FE1CE0101960E94BF05C12CC2
:101E2000D12C760159C0853789F402EE13E00E9467
:101E30005C03D8018D938D01B3E00D3F1B07B9F70B
:101E400061E080E00E94C9075AA241C08636B9F419
:101E50004982EBE4F3E0AE014D5F5F4F20813181B9
:101E60003296CA010197DC013C93DA012C934E5F54
:101E70005F4FB3E0EB36FB0789F761E2B3CF8736FC
:101E8000C9F40BE413E00E945C03682E0E945C031B
:101E9000262D30E0322F2227280F311DF801219303
:101EA00031938F01F3E00B361F0769F77AA20E9486
:101EB00063080DC0873481F4EBE4F3E011921192D2
:101EC00083E0EB36F807D1F70E9463087AA261E05D
:101ED000CE0182960E94BF0583E08093B6030E94E4
:101EE0003D0519CFA296E2E10C943A211F93CF93BE
:101EF000DF93C82FD62F61E00E941D1C61E08C2F5C
:101F00000E94561C61E08D2F0E94561C8AE090E0D2
:101F10000E94AE1B8D2F0E94891C892B71F060E0FE
:101F20008C2F0E94561C8AE090E00E94AE1B8D2FE1
:101F30000E94891C11E0892B09F010E060E08C2FD1
:101F40000E941D1C60E08C2F0E94561C60E08D2FAB
:101F50000E94561C812FDF91CF911F91089580E43C
:101F60008093BA001092BD008DE990E09093AE038B
:101F70008093AD031092480315E004E0C2E0FC2E0C
:101F800080914803813039F480E00E946204F0922D
:101F900048032D98F5CFC0914803C33061F42C98C5
:101FA00080918A030E948403C093B6030E943D057A
:101FB00000934803E5CF80914803843009F780916E
:101FC000B6038430E9F68FE70E944903C8EFD2E0F8
:101FD000E091E103E770F0E0EA56FD4F808190E088
:101FE0009E01285F32402817390724F40E945C03C1
:101FF0008993EECF109348032C9AC2CFAAE2B0E0A7
:10200000E4E0F0E10C942D211FEF198389E2E9EB64
:10201000F3E0DE01129601900D928A95E1F721E03E
:102020004AE2BE016F5F7F4F80E20E94540A811135
:102030000EC021E041E0BE016F5F7F4F80E20E9451
:10204000A90A811104C082E08093480302C0109362
:10205000480380914803823051F00E94591B6093DD
:102060004403709345038093460390934703AA96D5
:10207000E3E00C944921A1E0B0E0E1E4F0E10C944C
:102080002E21809148038230D9F480918A03805AAE
:10209000898321E041E0BE016F5F7F4F80E20E94B3
:1020A000540A882369F08FEF809348030E94591BDC
:1020B00060934403709345038093460390934703D2
:1020C0002196E2E00C944A21A1E0B0E0EAE6F0E1DA
:1020D0000C942E21809148038230D1F421E041E01C
:1020E000BE016F5F7F4F80E20E94A90A882371F0D2
:1020F0008FEF809348030E94591B609344037093B1
:102100004503809346039093470302C0898101C031
:102110008FEF2196E2E00C944A21A2E2B0E0E3E9DD
:10212000F0E10C941E219E012F5F3F4F80E1D90109
:102130001D928A95E9F768EE71E08AE094E029A3A0
:102140003AA30E94271D0E9460051D8A1E8A1F8ACD
:10215000188E312C212C00E0812C912C5401412C23
:1021600084E7582E8BE8682E82E3782E90E5C92EFE
:1021700093ECD92EE12CF12C84EF91E0A0E0B0E0BB
:102180008D8F9E8FAF8FB8A380E09EECADEEB4E351
:10219000898F9A8FAB8FBC8F80E094E7ABE8B2E376
:1021A000898B9A8BAB8BBC8B8AE094E00E94F31DE9
:1021B000892B09F4E1C08AE094E00E94201E9C0172
:1021C00033272C32310509F442C0ACF423323105F7
:1021D00009F0ABC019821A821B821C821D821E82EA
:1021E0001F82188619861A861B861C861D861E86E7
:1021F0001F86188A60C02434310529F02335310543
:1022000009F4B2C092C064E48AE094E00E940B1D1D
:102210002AE030E040E054E76BE872E38AE094E0C3
:102220000E94871D6CE28AE094E00E940B1D2AE068
:1022300030E040E05EEC6DEE74E38AE094E00E94F2
:10224000871D6CE28AE094E00E94391DADCF0F5FDC
:10225000043009F0A9CF29813A814B815C81A8EE35
:10226000B3E00E949A20698B7A8B8B8B9C8B2D819B
:102270003E814F8158850E949A20698F7A8F8B8F7B
:102280009C8F29853A854B855C852D8F3E8F4F8F9E
:1022900058A32D853E854F8558890E949A206B0151
:1022A0007C0160323EE473078105910530F462E3FE
:1022B0008CE10E94710300E077CF603345E774073B
:1022C0008105910510F462E2F3CF60345CE9750793
:1022D0008105910510F466E2EBCF80E5C81683EC2A
:1022E000D806E104F10410F462E1E2CF90E6C916E9
:1022F0009AEED906E104F10410F465E1D9CFA0E724
:10230000CA16A1E1DA06A1E0EA06F10410F461E0E0
:10231000CFCFB0EACB16B6E8DB06B1E0EB06F104AE
:1023200010F463E0C5CF65E0C3CF10ED180F1A308D
:1023300008F03ACFE1E0F0E0EC0FFD1F24E0029F4F
:10234000E00DF11D11242081318142815381AAE0E9
:10235000B0E00E949A20610F711D811D911D608364
:1023600071838283938320CF49885A886B887C88C5
:10237000812C912C540118CF81149104A104B10433
:1023800089F4C301B2010E94F70361E070E080E0CC
:1023900090E00E94881B1D8A1E8A1F8A188E312C8D
:1023A00022242A948D8D9E8DAF8DB8A18816990612
:1023B000AA06BB06D0F40E949A032D893E894F8954
:1023C000588D280F311D411D511D2D8B3E8B4F8B7C
:1023D000588F381608F4382E821508F4282E3FEF4F
:1023E000831A930AA30AB30A56C0C301B20128EEA6
:1023F00033E040E050E00E94DD20BA01A9012AE06C
:1024000030E08AE094E00E94D51D6CE28AE094E01E
:102410000E940B1D4AE050E0632D8AE094E00E9488
:10242000E41D6CE28AE094E00E940B1D6D897E89B8
:102430008F89988DA50194010E94DD20BA01A90120
:102440002AE030E08AE094E00E94D51D6CE28AE048
:1024500094E00E940B1D4AE050E0622D8AE094E077
:102460000E94E41D6CE28AE094E00E94391D4C0C4D
:102470005D1C6E1C7F1C898D9A8DAB8DBC8D841567
:102480009505A605B70520F449885A886B887C888D
:10249000812C912C540129893A894B895C89283EE9
:1024A00033404105510509F07FCEA296E2E10C943C
:1024B0003A21A1E0B0E0EFE5F2E10C942E2180E0BA
:1024C0000E948E0161E08CE00E941D1C61E08DE0A5
:1024D0000E941D1C0E94650160E080E00E941D1C9E
:1024E00061E081E00E941D1C40E052EC61E070E080
:1024F0008AE094E00E943B1F0E94B5080E94680891
:1025000065EF71E08AE094E00E94081D88E893E09E
:102510000E9464076CE072E08AE094E00E94081D6B
:102520004AE050E062E070E08AE094E00E94BD1D65
:102530000E947A0178942D9A62E18EE00E94760FD3
:10254000882329F02D982C980E948D10FBCF63E0F2
:102550008AE00E94760F811104C00E945108811107
:1025600019C06FE472E08AE094E00E94081D60E008
:1025700070E0CB010E94670E882349F00E945E083C
:1025800064E172E08AE094E00E94271D2C9A0E9488
:102590004E0D10C00E944E0D8091E603823209F06C
:1025A000C6C08091E703833209F0C1C08091F00377
:1025B00081FDC3C08091E603823231F58091E7034B
:1025C000833211F581E00E94BF088091F00382FF01
:1025D00008C06FE272E08AE094E00E94271D0E942A
:1025E000AF0F64E170E080E090E00E94881B21E082
:1025F00041E0BE016F5F7F4F80E20E94A90A811116
:1026000003C081E0809348036AE372E08AE094E0CB
:102610000E94081D8FE00E948E0180E00E946204EB
:1026200010928A0380E00E94840380E0883170F079
:102630008093CC0283E08093B6030E946005809172
:102640004803882371F00E94FE0F0BC021E0280F81
:10265000E82FF0E0E754FC4F9785992349F3822F48
:10266000E5CF8091E903982F9D7F983229F440E0CF
:1026700052EC61E070E023C0893251F42EE240EA6E
:1026800056E861E070E08AE094E00E94BC1F1BC045
:102690008091E1038871803129F440E855E260E0DF
:1026A00070E00DC04091BA035091BB036091BC0330
:1026B0007091BD034A3051056105710570F38AE0E0
:1026C00094E00E943B1F8AE094E00E94F31D892B56
:1026D00029F08AE094E00E94201EF5CF8091E80363
:1026E000843229F08091C1008F7E8093C100809157
:1026F000E903853241F08852833028F08091C1008F
:10270000877F8093C1001092CE021092CD0210926A
:102710004A030E94651B609386037093870380932E
:102720008803909389032196E2E00C944A218091DA
:10273000F0038B7F8093F00339CF82FD3BCF64EFB2
:1027400071E080E090E00E94670E882309F432CFA8
:102750000E945E0864E172E08AE094E00E94271D16
:102760000E944E0D2C9A26CFCF93DF938AE094E0FF
:102770000E94F31D892BE9F0C091CD02D0E0CE017B
:1027800001968F7199272091CE0230E0821793072E
:1027900081F08AE094E00E94201EC153DD4F8883BF
:1027A0008091CD0290E001968F7199278093CD02A0
:1027B000DDCFDF91CF910895A0E0B0E0E2EEF3E14C
:1027C0000C942821D82FC62F0E94651B0091A303CB
:1027D0001091A4032091A5033091A6036B017C0105
:1027E000C01AD10AE20AF30A9701860141E1C41630
:1027F00047E2D406E104F10408F4D1C16093A303D5
:102800007093A4038093A5039093A60380910D0178
:1028100090910E01880F991F80938B03892F8770E9
:1028200020918C03287F282B20938C0380910F010B
:1028300090911001880F991F382F330F330F330FEA
:102840002770232B20938C03282F22952695277001
:1028500080918D03807C9770990F990F990F822B2F
:10286000892B80938D032091110130911201220F49
:10287000331F922F9295990F990F907C8F73892B0C
:1028800080938D03932F9295990F990F907C822FAF
:1028900086958695892B80938E0332FB882780F955
:1028A00020918F032E7F282B20938F03809113017B
:1028B00090911401880F991F382F330F2170232B0B
:1028C00020938F03382F331F3327331F209190031A
:1028D000207F892F8770880F232B282B209390032C
:1028E0008091150190911601880F991F382F32950C
:1028F000307F2F70232B20939003382F32953F7019
:10290000209191032078892F87708295807F232BD7
:10291000282B209391038091170190911801880F23
:10292000991F2F7720939103292F279522272795E9
:102930008695822B80939203892F869583702091B0
:1029400093032C7F282B209393038091190190915E
:102950001A01880F991F382F330F330F2370232B41
:1029600020939303382F3295369536953370209106
:102970009403207E892F8770880F880F232B282BA4
:102980002093940380911B0190911C01880F991F43
:10299000382F3295330F307E2F71232B20939403E1
:1029A0009295990F907E869586958695892B809332
:1029B000950380911D0190911E01880F991F8093AE
:1029C0009603892F877020919703287F282B2093C7
:1029D000970380911F0190912001880F991F382F34
:1029E000330F330F330F2770232B20939703282F98
:1029F00022952695277080919803807C9770990F77
:102A0000990F990F822B892B809398032091210194
:102A100030912201220F331F922F9295990F990F17
:102A2000907C8F73892B80939803932F9295990FA5
:102A3000990F907C822F86958695892B8093990398
:102A400032FB882780F920919A032E7F282B209330
:102A50009A038091230190912401880F991F382FA8
:102A6000330F2170232B20939A03382F331F3327E2
:102A7000331F20919B03207F892F8770880F232B82
:102A8000282B20939B038091250190912601880F8C
:102A9000991F382F3295307F2F70232B20939B0363
:102AA000382F32953F7020919C032078892F8770B2
:102AB0008295807F232B282B20939C0380912701D4
:102AC00090912801880F991F2F7720939C03292F1D
:102AD0002795222727958695822B80939D0396958F
:102AE000937080919E038C7F892B80939E0320910D
:102AF000290130912A01220F331F922F990F990F2C
:102B00008370892B80939E032295269526952370AA
:102B100080919F03807E932F9770990F990F822B3E
:102B2000892B80939F0320912B0130912C01220F40
:102B3000331F922F9295990F907E8F71892B8093DE
:102B40009F03832F8295880F807E26952695269554
:102B5000282B2093A003DD2311F088E001C080E042
:102B6000CC2311F094E001C090E0892B8093A10365
:102B70006FE070E08AE094E00E940201CBE8D3E0CD
:102B800069918AE094E00E944D1E83E0C23AD80722
:102B9000B9F760E070E08AE094E00E940201CDB7EE
:102BA000DEB7E8E00C944421CF93C82F682F8AE069
:102BB00094E00E944D1E8C2F0E940A01CF9108952F
:102BC000A0E0B0E0E6EEF5E10C942821C82F0E94C9
:102BD000651B0091A3031091A4032091A5033091DC
:102BE000A6036B017C01C01AD10AE20AF30A97011D
:102BF000860141E1C41647E2D406E104F10408F479
:102C000045C06093A3037093A4038093A50390939E
:102C1000A6031092B8031092B70388EA0E94D41555
:102C2000CC2311F081E801C081E00E94D41580E13D
:102C30000E94D41500E010E0F801EE0FFF1FE35FE3
:102C4000FE4F808191810E94DB02EC01B3E0CC0F4A
:102C5000DD1FBA95E1F78D2F0E94D4158C2F0E94AD
:102C6000D4150F5F1F4F0031110531F76091B80384
:102C700070E08AE094E00E94FA006091B7037091DE
:102C8000B80377278AE094E00E94FA00CDB7DEB758
:102C9000E8E00C944421AAE1B0E0E1E5F6E10C940F
:102CA00020210E949B008CE00E946B0381110BC0CD
:102CB00068E872E08AE094E00E94271D80E00E94AC
:102CC00062040E9460050E94B4130E94651B0E946A
:102CD000641091E0853009F090E01FEF8091B60319
:102CE000843009F4FEC19111FCC17CC00E949E0396
:102CF00090937303809372032C9AC0928603D092B0
:102D00008703E0928803F09289031092490380912F
:102D1000700390917103880F991F816090937103E4
:102D2000809370032D9880E00E944E0E8091F802EF
:102D3000982F9E7309F02CC2F8948091E10349EF1B
:102D400052E06DE071E087700E942A020E94680CD8
:102D500078949091F8028091420390FF13C2811100
:102D600024C09BE4E92E93E0F92E00E010E0F70187
:102D70008081918194FD0CC0F801EE0FFF1FE35F8D
:102D8000FE4F808191810E94DB02D7018D939C933D
:102D90000F5F1F4FB2E0EB0EF11C0031110539F748
:102DA0000E94630881E08093420380914A0381116D
:102DB00003C081E080934A0310926B0310926D036D
:102DC00010926C038091E103887109F009C20E949E
:102DD000DC0C83E08093B6030E943D0581E0809384
:102DE00043032C980E94651B4B015C010E94591BF8
:102DF0006B017C0180914903823008F063C04090F0
:102E000086035090870360908803709089038091B7
:102E1000820390918303A0918403B091850384156C
:102E20009505A605B70509F44DC089EB93E00E940E
:102E3000B8016C5D754081099109950184010419FF
:102E40001509260937096017710782079307D0F51E
:102E500040928203509283036092840370928503B0
:102E60000E949A03282F8093760380917703909194
:102E70007803820F911D909378038093770360917C
:102E800079036F5F609379036930E0F070E00E942E
:102E9000C920709378036093770380917503E3E012
:102EA0008E9F600D711D11247695679576956795B7
:102EB000609375030E94A10C10927803109277031F
:102EC0001092790380914A030091CC02882351F13A
:102ED00010914903101708F029C2409086035090C2
:102EE00087036090880370908903A50194012419D9
:102EF0003509460957092F8B388F498F5A8F89EB2F
:102F000093E00E94B80168517C4F8F4F9F4F2F89EB
:102F1000388D498D5A8D621773078407950708F419
:102F2000CCC104C28091860390918703A09188034D
:102F3000B091890375016401C81AD90AEA0AFB0A2B
:102F400089EB93E00E94B8019B01AC01A02FB0E097
:102F50000E949A206C157D058E059F0558F480927D
:102F6000860390928703A0928803B092890381E040
:102F70008093430380916C03811116C08091E90313
:102F8000883219F40E94000B0FC0893239F4609125
:102F9000490380916B030E94DC1306C08A3221F43E
:102FA00080916B030E94E01580914303882309F40C
:102FB00072C0E0918A03EF5FE0938A03E83131F059
:102FC000F0E0E754FC4F8785811102C010928A031C
:102FD0008091F2039091F303A091F403B091F50373
:102FE000892B8A2B8B2B09F44EC080917A03909108
:102FF0007B03A0917C03B0917D03892B8A2B8B2BC3
:1030000009F441C00E945006082F10E020910901E8
:1030100030910A0136952795369527952C5E3F4FBE
:103020002017310770F40E94591B68517C4F8F4F55
:103030009F4F60937A0370937B0380937C039093FC
:103040007D03C801880F991F880F991F40910901BE
:1030500050910A019A01220F331F240F351F820F4E
:10306000931F969587959695879590930A018093DF
:1030700009016091BE037091BF038091C0039091DC
:10308000C1030E94F70380918A030E9484030E9477
:103090003B1010924303809148038F3F09F041C2D7
:1030A0000E94591B0091440310914503209146034F
:1030B00030914703601B710B820B930B693E734089
:1030C0008105910508F42DC20E94591B60934403A9
:1030D0007093450380934603909347030E94FE0F2D
:1030E00020C20E94651B6B017C018091B603843075
:1030F000D1F48FE70E94490308EF12E0E091E10369
:10310000E770F0E0EA56FD4F808190E09801285F7B
:103110003240281739070CF0E9CD0E945C03D80132
:103120008D938D01EBCFE091E103E770F0E0EA567B
:10313000FD4F40814F5F21E0BE016F5F7F4F80E216
:103140000E94A90A882371F0109348030E94591B1A
:103150006093440370934503809346039093470321
:1031600090E0BCCDE091E103E770F0E0EA56FD4F5E
:10317000408150E0BE016E5F7F4F88EF92E00E9479
:103180005B21BBCD882309F410CE109242030DCEF3
:10319000982F9873983309F008CE9091EF02892701
:1031A00087FF03CE90589093EF028091E903853218
:1031B00009F0FBCD10E0212F30E08091F8028770FC
:1031C00090E0821793070CF4F0CD1F5FE12FF0E041
:1031D000E850FD4F60818AE094E00E944D1EEBCFE5
:1031E0008091EF029091F802982796FD5AC0807C5A
:1031F00090E489278093EF028091CE023091CD0236
:103200008317D1F0E0EFF2E020E02F5F90E0DC01E7
:10321000A153BD4F4C91419301968F71992728304E
:1032200011F08313F2CF8093CE02295C8091EF02DC
:10323000282B2093EF0235C0809176038093F00213
:103240008091E603863251F482E10E94B21C95958A
:103250008795959587958093F10202C01092F102AF
:103260008091E703863251F483E10E94B21C959568
:103270008795959587958093F20202C01092F2028D
:1032800080917203909173039093F3028093F40200
:1032900080917003909171039F770E94FC0280934C
:1032A000F50269E08FEE92E00E9478050E94E70542
:1032B00081118DCD0E94B413F9CF8091700390914C
:1032C0007103880F991F909371038093700381E0BD
:1032D00080934303111110C0C0927E03D0927F03EC
:1032E000E0928003F092810310927A0310927B03A4
:1032F00010927C0310927D031F5F1093490389EBAA
:1033000093E00E94B801640D751D861D971D6093A2
:1033100086037093870380938803909389032D9A83
:1033200081E00E944E0E0E94A10C03C0101709F408
:10333000A7C080914903882309F41CCE8091FA0329
:103340008823D9F090916B03911117C040917E03AF
:1033500050917F0360918003709181034601570172
:10336000841A950AA60AB70A90E00E9423016815FC
:1033700079058A059B0508F4B5C08091FC03882374
:10338000D9F090916D03911117C040917E03509137
:103390007F03609180037091810346015701841A75
:1033A000950AA60AB70A90E00E94230168157905DC
:1033B0008A059B0508F4ADC08091FB038823D9F0F2
:1033C00090916C03911117C040917E0350917F033F
:1033D000609180037091810346015701841A950A18
:1033E000A60AB70A90E00E942301681579058A05AC
:1033F0009B0508F492C08091F2039091F303A09191
:10340000F403B091F503892B8A2B8B2B09F4B2CDF1
:1034100080917A0390917B03A0917C03B0917D030E
:103420000097A105B10509F4A5CDC81AD90AEA0A81
:10343000FB0AF7FC9FCD8091F003829581700E947A
:10344000930680E00E9462040E943D050E94591B81
:103450006B017C012091F70330E0A8EEB3E00E94FD
:103460008B20C60ED71EE81EF91E6894C0F8C092C5
:103470007A03D0927B03E0927C03F0927D037ACDB5
:103480008091860390918703A0918803B09189036E
:1034900024013501481A590A6A0A7B0A89EB93E02C
:1034A0000E94B8019B01AC01A12FB0E00E949A20BC
:1034B000641575058605970508F03BCF10927103DA
:1034C0001092700381E080934303109275030E9471
:1034D000A10C8092860390928703A0928803B092F9
:1034E000890327CF81E080936B030E94160D8091A2
:1034F000F6030E9448016C0D7D1D8E1D9F1D6160AD
:1035000060937A0370937B0380937C0390937D0395
:1035100034CF81E080936D034FCF81E080936C03C3
:103520006ACF6A96E0E10C943C218230E8F4E82FFF
:10353000F0E0EE0FFF1FE350FC4F7183608381309A
:1035400041F0809169008C7F842B80936900E89A18
:10355000089580916900440F551F440F551F837FC4
:10356000842B80936900E99A08951F920F920FB6F9
:103570000F9211242F933F934F935F936F937F93F9
:103580008F939F93AF93BF93EF93FF938091FD032E
:103590009091FE03892B29F0E091FD03F091FE0349
:1035A0000995FF91EF91BF91AF919F918F917F917D
:1035B0006F915F914F913F912F910F900FBE0F90A0
:1035C0001F9018951F920F920FB60F9211242F93F0
:1035D0003F934F935F936F937F938F939F93AF939B
:1035E000BF93EF93FF938091FF0390910004892B89
:1035F00029F0E091FF03F09100040995FF91EF910C
:10360000BF91AF919F918F917F916F915F914F91FA
:103610003F912F910F900FBE0F901F9018951F9202
:103620000F920FB60F9211242F933F938F939F9376
:10363000AF93BF938091020490910304A09104047E
:10364000B09105043091010423E0230F2D3720F4BD
:103650000196A11DB11D05C026E8230F0296A11DEC
:10366000B11D209301048093020490930304A0935E
:103670000404B09305048091060490910704A0917E
:103680000804B09109040196A11DB11D80930604A0
:1036900090930704A0930804B0930904BF91AF91DD
:1036A0009F918F913F912F910F900FBE0F901F9080
:1036B00018952FB7F89460910204709103048091DB
:1036C0000404909105042FBF08953FB7F8948091AA
:1036D000060490910704A0910804B091090426B54E
:1036E000A89B05C02F3F19F00196A11DB11D3FBF3A
:1036F0006627782F892F9A2F620F711D811D911DCA
:1037000042E0660F771F881F991F4A95D1F70895E9
:10371000CF92DF92EF92FF92CF93DF936B017C0108
:103720000E94651BEB01C114D104E104F10479F09E
:103730000E94651B6C1B7D0B683E7340A0F381E00B
:10374000C81AD108E108F108C851DC4FECCFDF916D
:10375000CF91FF90EF90DF90CF9008950197009761
:1037600039F0880F991F880F991F02970197F1F779
:103770000895789484B5826084BD84B5816084BDE9
:1037800085B5826085BD85B5816085BDEEE6F0E0DA
:10379000808181608083E1E8F0E010828081826036
:1037A0008083808181608083E0E8F0E080818160B7
:1037B0008083E1EBF0E0808184608083E0EBF0E0E7
:1037C000808181608083EAE7F0E08081846080838B
:1037D0008081826080838081816080838081806835
:1037E00080831092C1000895833081F028F48130E5
:1037F00099F08230A1F008958630A9F08730B9F0B1
:103800008430D1F4809180008F7D03C0809180004E
:103810008F7780938000089584B58F7702C084B538
:103820008F7D84BD08958091B0008F7703C0809113
:10383000B0008F7D8093B0000895CF93DF9390E028
:10384000FC01E458FF4F2491FC01E057FF4F8491A5
:10385000882349F190E0880F991FFC01E854FF4F3D
:10386000A591B49182559F4FFC01C591D4919FB70A
:10387000611108C0F8948C91209582238C938881E3
:1038800082230AC0623051F4F8948C91322F309523
:1038900083238C938881822B888304C0F8948C9135
:1038A000822B8C939FBFDF91CF910895A1E0B0E070
:1038B000ECE5FCE10C942C21282F30E0F901E859CB
:1038C000FF4F8491F901E458FF4F1491F901E0573B
:1038D000FF4F04910023C9F0882321F069830E94DF
:1038E000F41B6981E02FF0E0EE0FFF1FE255FF4F60
:1038F000A591B4919FB7F8948C91611103C0109574
:10390000812301C0812B8C939FBF2196E4E00C940E
:103910004821CF93DF93282F30E0F901E859FF4F7A
:103920008491F901E458FF4FD491F901E057FF4F1A
:10393000C491CC2391F081110E94F41BEC2FF0E094
:10394000EE0FFF1FEC55FF4FA591B4912C912D2345
:1039500081E090E021F480E002C080E090E0DF911F
:10396000CF9108958E3008F08E5087702091B90164
:1039700090E4299F90011124822B80937C008091F8
:103980007A00806480937A0080917A0086FDFCCF73
:10399000809178002091790090E0922B0895A0E02A
:1039A000B0E0E5EDFCE10C9428216C017A01EB011B
:1039B000E60EF71E00E010E0CE15DF0561F069911C
:1039C000D601ED91FC910190F081E02DC6010995A1
:1039D000080F191FF1CFC801CDB7DEB7E8E00C948E
:1039E00044216115710589F0DB010D900020E9F794
:1039F000AD0141505109461B570BDC01ED91FC9183
:103A00000280F381E02D0995089580E090E008950B
:103A10000E94F11C0895DC01ED91FC910190F08170
:103A2000E02D099508950F931F93CF93DF93EC0139
:103A30006DE00E940B1D8C016AE0CE010E940B1DFF
:103A4000800F911FDF91CF911F910F9108950F93D8
:103A50001F93CF93DF93EC010E94F11C8C01CE01E8
:103A60000E94131D800F911FDF91CF911F910F9125
:103A700008950F931F93CF93DF93EC010E940B1DCA
:103A80008C01CE010E94131D800F911FDF91CF91F9
:103A90001F910F910895A1E2B0E0E1E5FDE10C94E2
:103AA00024217C01C42EE52FCB01D22E19A221E0C6
:103AB0002D1510F02AE0D22E8E010F5D1F4F8D2C98
:103AC000912CA12CB12C6C2D7E2FA50194010E946C
:103AD000DD208C2DD29E80191124015011098A30CD
:103AE00010F4805D01C0895CF801808321153105E7
:103AF0004105510521F0C22EE32FCA01E4CFB801E0
:103B0000C7010E94F11CA196ECE00C944021A0E0BA
:103B1000B0E0EDE8FDE10C942821EC016A017B01A5
:103B20002115310541F4E881F9810190F081E02D02
:103B3000642F09951DC02A303105A9F477FF12C002
:103B40006DE20E940B1D8C0144275527BA014C19C8
:103B50005D096E097F092AE0CE010E944B1D800F8E
:103B6000911F06C02AE0B701A601CE010E944B1D9D
:103B7000CDB7DEB7E8E00C9444210F931F93CF93A9
:103B8000DF93EC019A01AB01662757FD6095762F14
:103B90000E94871D8C01CE010E94131D800F911F72
:103BA000DF91CF911F910F9108952115310549F4AF
:103BB000DC01ED91FC910190F081E02D642F0995DD
:103BC00008950E944B1D08959A01462F50E060E031
:103BD00070E00E94D51D08959A01AB0160E070E08D
:103BE0000E94D51D0895FC0124853585F901E05C0E
:103BF000FF4F80819181F901EE5BFF4F2081318180
:103C0000821B930B8F7399270895FC0184859585FA
:103C1000FC01E05CFF4F40815181FC01EE5BFF4FF6
:103C2000208131814217530741F00190F081E02D4E
:103C3000E80FF91F808190E008958FEF9FEF0895BE
:103C4000FC0184859585FC01E05CFF4F408151813A
:103C5000FC01EE5BFF4F208131814217530779F061
:103C6000A081B181A80FB91F8C91208131812F5F74
:103C70003F4F2F7333273183208390E008958FEFD8
:103C80009FEF0895FC0181A1882329F0A489B589BB
:103C90008C9186FFFBCF11A20895CF93DF93FC0197
:103CA00026853785D901A05CBF4F8D919C911197D6
:103CB00001968F739927E901CE5BDF4F48815981C7
:103CC00084179507D9F30D90BC91A02DA20FB31FB7
:103CD0006C93A685B785A05CBF4F11969C938E937D
:103CE000A689B7892C9181E090E0078C02C0880FEB
:103CF000991F0A94E2F7282B2C9381E081A3048872
:103D0000F589E02D80818064808381E090E0DF91FF
:103D1000CF91089508951F920F920FB60F9211241C
:103D20002F933F934F938F939F93EF93FF938091A4
:103D3000C00082FD1CC04091C6008091B0049091EB
:103D4000B10401968F7399272091B2043091B30486
:103D50008217930771F0E091B004F091B104E0593B
:103D6000FB4F40839093B1048093B00402C08091D4
:103D7000C600FF91EF919F918F914F913F912F91AD
:103D80000F900FBE0F901F9018958AE094E00E944C
:103D9000F31D892B11F00E948A1E08951F920F9225
:103DA0000FB60F9211242F933F938F939F93EF930E
:103DB000FF9320916C0430916D0480916E0490917A
:103DC0006F042817390731F48091C1008F7D8093EB
:103DD000C10014C0E0916E04F0916F04E45DFB4FEC
:103DE000208180916E0490916F0401968F739927C2
:103DF00090936F0480936E042093C600FF91EF911F
:103E00009F918F913F912F910F900FBE0F901F9018
:103E10001895A0E0B0E0EFE0FFE10C942421FC0154
:103E20001382128288EE93E0A0E0B0E08483958351
:103E3000A683B7838EEB92E0918380837587648736
:103E400057874687318B208B138B028BF58AE48A48
:103E5000D78AC68AB18EA08E938E828E8F85848FEC
:103E60008889858F8989868F8A89878F8B8980A3A6
:103E7000ECE00C944021CF92DF92EF92FF92CF932F
:103E8000DF93EC016A017B01411581EE5807610562
:103E90007105F9F0EC89FD8981E090E008A002C08D
:103EA000880F991F0A94E2F7808360E079E08DE340
:103EB00090E0A70196010E94DD20215031094109BF
:103EC00051095695479537952795211580E1380773
:103ED00098F0EC89FD89108260E874E88EE190E04A
:103EE000A70196010E94DD202150310941095109A5
:103EF0005695479537952795E889F9893083EA895A
:103F0000FB89208319A2EE89FF89408181E090E03E
:103F10009C010C8C02C0220F331F0A94E2F7422B43
:103F20004083EE89FF8940819C010D8C02C0220FE5
:103F3000331F0A94E2F7422B4083EE89FF894081C8
:103F40009C010E8C02C0220F331F0A94E2F7422B11
:103F50004083EE89FF8920810F8C02C0880F991F52
:103F60000A94E2F7809582238083DF91CF91FF90BE
:103F7000EF90DF90CF900895BF92CF92DF92EF92B3
:103F8000FF92CF93DF93EC016A017B01B22E4115C2
:103F900081EE580761057105F9F0EC89FD8981E032
:103FA00090E008A002C0880F991F0A94E2F780836E
:103FB00060E079E08DE390E0A70196010E94DD20AA
:103FC0002150310941095109569547953795279553
:103FD000211580E1380798F0EC89FD89108260E8AE
:103FE00074E88EE190E0A70196010E94DD20215047
:103FF0003109410951095695479537952795E88923
:10400000F9893083EA89FB892083E88DF98DB082B4
:10401000EE89FF89408181E090E09C010C8C02C018
:10402000220F331F0A94E2F7422B4083EE89FF8967
:1040300040819C010D8C02C0220F331F0A94E2F7CD
:10404000422B4083EE89FF8940819C010E8C02C087
:10405000220F331F0A94E2F7422B4083EE89FF8937
:1040600020810F8C02C0880F991F0A94E2F7809577
:1040700082238083DF91CF91FF90EF90DF90CF90EC
:10408000BF9008958F929F92AF92BF92CF92DF928E
:10409000EF92FF920F931F9381E08F9385E08F93B0
:1040A00087E08F9383E08F9384E08F93E6EC8E2EEE
:1040B000912CF2ECAF2EB12CA1ECCA2ED12CB0EC8D
:1040C000EB2EF12C04EC10E025EC30E04CE254E057
:1040D00060E774E08AE094E00E94091F0F900F905F
:1040E0000F900F900F901F910F91FF90EF90DF9026
:1040F000CF90BF90AF909F908F9008950E94B91B72
:104100000E945912C5ECDEE10E944B162097E1F3A4
:104110000E94C51EF9CFA29FB001B39FC001A39F0B
:10412000700D811D1124911DB29F700D811D1124F0
:10413000911D08950E948B20A59F900DB49F900D16
:10414000A49F800D911D11240895B7FF0C949A200F
:104150000E949A20821B930B0895DB018F939F93FB
:104160000E949A20BF91AF91A29F800D911DA39FA5
:10417000900DB29F900D11240895991B79E004C011
:10418000991F961708F0961B881F7A95C9F7809596
:104190000895AA1BBB1B51E107C0AA1FBB1FA6178E
:1041A000B70710F0A61BB70B881F991F5A95A9F7E0
:1041B00080959095BC01CD010895A1E21A2EAA1B0D
:1041C000BB1BFD010DC0AA1FBB1FEE1FFF1FA217C7
:1041D000B307E407F50720F0A21BB30BE40BF50BC4
:1041E000661F771F881F991F1A9469F7609570954D
:1041F000809590959B01AC01BD01CF010895052EDE
:1042000097FB1EF400940E94162157FD07D00E94D0
:10421000DD2007FC03D04EF40C94162150954095F8
:10422000309521953F4F4F4F5F4F08959095809562
:10423000709561957F4F8F4F9F4F08952F923F92BA
:104240004F925F926F927F928F929F92AF92BF92A6
:10425000CF92DF92EF92FF920F931F93CF93DF9352
:10426000CDB7DEB7CA1BDB0B0FB6F894DEBF0FBEAF
:10427000CDBF09942A88398848885F846E847D84FC
:104280008C849B84AA84B984C884DF80EE80FD80FE
:104290000C811B81AA81B981CE0FD11D0FB6F89474
:1042A000DEBF0FBECDBFED010895EE0FFF1F0590DD
:1042B000F491E02D0994FB01DC0102C001900D9204
:1042C00041505040D8F70895F999FECF92BD81BD75
:1042D000F89A992780B50895262FF999FECF1FBA2D
:1042E00092BD81BD20BD0FB6F894FA9AF99A0FBE1F
:0842F00001960895F894FFCF38
:1042F8000000B404200008409CFF0088130002005E
:104308000200020002000200020002000200020095
:104318000200020002000200020002000200200166
:10432800270121022B032203260423042605240641
:104338002506280629062A8025000005400AA1200E
:104348004EA50020244EA52C2330C01200001A4090
:104358000AA1204EA5001B1E27522C2330802500C1
:104368000005400AA1204EA50020244EA52C23308C
:10437800004B000006400AD0009D49007B289D495B
:104388002C233000E1000005400A4501D7DC03B8C2
:104398001E0EBF00232E48E801008A400A6001551E
:1043A8005502AD1E20000023C80154582074696DC1
:1043B800656F7574210057616974696E6720626959
:1043C8006E640A00476F7420706B740A006461742D
:1043D8006120676F6F640A007363616E6E65722097
:1043E8006D6F6465004F70656E4C52536E67205256
:1043F80058207374617274696E672000206F6E2094
:104408004857200053617665642062696E642064B1
:1044180061746120746F20454550524F4D0A004920
:1044280020616D20736C61766500456E74657269F4
:104438006E67206E6F726D616C206D6F64650045EC
:104448004550524F4D2064617461206E6F74207620
:10445800616C6964206F722062696E64206A756D90
:1044680070706572207365742C20666F7263696E54
:10447800672062696E640A0052582068616E67009E
:10448800B200F4014C0300070B0C101115000A03CD
:104498000E121300010400000000080001000010C3
:1044A80000002000000001000002000000004D1E76
:0A44B800CF1CF31D201E051E421E3E
:107E00000F92CDB7DEB7112484B714BE81FFF1D035
:107E100082E08093C00088E18093C10086E0809377
:107E2000C20080E18093C4008EE0CDD088249924E4
:107E3000CC24C394F5E0DF2EE1E1EE2E73E0F72EC3
:107E4000B6D0082F813479F4B2D08983C2D0898129
:107E5000823811F481E005C0813811F485E001C059
:107E600083E09ED09AC0823411F484E103C085344B
:107E700019F485E0B6D091C0853561F498D0082F0B
:107E800010E095D090E0982E8824802A912A880CC2
:107E9000991C82C0863521F484E0A3D080E0E1CF34
:107EA000843609F04CC083D082D0A82E80D0B82E62
:107EB00000E011E07CD0F80181938F01AE16D1F77C
:107EC00088D0FB2DF53489F4E0E0F1E00BC0F9999E
:107ED000FECF92BC81BC0894811C911C819180BD15
:107EE000FA9AF99AEA1598F358C08B2D863409F05E
:107EF00054C0F401F7BEE89507B600FCFDCFF401CD
:107F0000A0E0B1E02C9130E011968C91119790E0B7
:107F1000982F8827822B932B12960C01C7BEE895C9
:107F20001124329681E0A038B80761F7F401D7BE7A
:107F3000E89507B600FCFDCFE7BEE8952EC0843774
:107F4000F1F435D034D0182F32D0B82E42D0FB2DDA
:107F5000F63421F4F40105914F010CC0FB2DF534EA
:107F600049F4F999FECF92BC81BC0894811C911C04
:107F7000F89A00B5802F14D0115049F70EC08537FC
:107F800039F427D08EE10CD085E90AD08FE069CF93
:107F9000813511F488E017D01CD080E101D050CF9A
:107FA0009091C00095FFFCCF8093C600089580910A
:107FB000C00087FFFCCF8091C00084FD01C0A89560
:107FC0008091C6000895E0E6F0E098E19083808318
:107FD0000895EDDF803219F088E0F5DFFFCF84E10E
:107FE000DFCF1F93182FE3DF1150E9F7F2DF1F9166
:0E7FF0000895282E80E0E7DFEE27FF27099492
:027FFE0001057B
:0400000300007E007B
:00000001FF
